:100000000A168A150028FF3FFF00030E8301DE0059
:100010000408DD000A08DF008A017C088316B300AB
:100020007B08B2007A08B1007008B0008312A00A01
:1000300002302002031C1D28A0010330FC00FF3009
:10004000FB00FF30FA00FC0B26282D28FB0B29288B
:100050002C28FA0B2928262823288C30FB00FF3077
:10006000FA00FB0B34283728FA0B34283128A1304A
:10007000FA00FA0B392800008B1083163308FC00B5
:100080003208FB003108FA003008F00083125F08E4
:100090008A005D0884005E0E8300FF0E7F0E09005B
:1000A000031383127408F8027508031C750FF90214
:1000B0007608031C760FFA027708031C770FFB0201
:1000C000F30D0730FC00730DF80DF90DFA0DFB0D63
:1000D0007408731C7928F8027508031C750FF9025F
:1000E0007608031C760FFA027708031C770FFB02D1
:1000F0008628F80775080318750FF907760803189E
:10010000760FFA0777080318770FFB07F30DFC0B40
:100110006328720DF80DF90DFA0DFB0D7408731CB0
:100120009F28F8027508031C750FF9027608031C56
:10013000760FFA027708031C770FFB02AC28F8074A
:1001400075080318750FF90776080318760FFA0774
:1001500077080318770FFB07F20D0730FC00720DCC
:10016000F80DF90DFA0DFB0D7408721CC528F80284
:100170007508031C750FF9027608031C760FFA0246
:100180007708031C770FFB02D228F80775080318BD
:10019000750FF90776080318760FFA077708031822
:1001A000770FFB07F20DFC0BAF28710DF80DF90D61
:1001B000FA0DFB0D7408721CEB28F8027508031C7D
:1001C000750FF9027608031C760FFA027708031CF4
:1001D000770FFB02F828F80775080318750FF90761
:1001E00076080318760FFA0777080318770FFB07CE
:1001F000F10D0730FC00710DF80DF90DFA0DFB0D36
:100200007408711C1129F8027508031C750FF90296
:100210007608031C760FFA027708031C770FFB029F
:100220001E29F80775080318750FF90776080318D3
:10023000760FFA0777080318770FFB07F10DFC0B11
:10024000FB28700DF80DF90DFA0DFB0D7408711CEB
:100250003729F8027508031C750FF9027608031C8C
:10026000760FFA027708031C770FFB024429F80780
:1002700075080318750FF90776080318760FFA0743
:1002800077080318770FFB07F00D0730FC00700D9F
:10029000F80DF90DFA0DFB0D7408701C5D29F802BC
:1002A0007508031C750FF9027608031C760FFA0215
:1002B0007708031C770FFB026A29F80775080318F3
:1002C000750FF90776080318760FFA0777080318F1
:1002D000770FFB07F00DFC0B472970187D29740878
:1002E000F80775080318750FF90776080318760FD5
:1002F000FA0777080318770FFB0708008A15BD2255
:100300008A118A15BD228A118A15BD228A11831687
:100310002508F00001308312A40070080319942905
:10032000A40D2410FF3F8E2983162608F00001300B
:100330008312A50070080319A129A50D2510FF3F00
:100340009B2983162708F00001308312A60070084D
:100350000319AE29A60D2610FF3FA82983162808E9
:10036000F00001308312A70070080319BB29A70D04
:100370002710FF3FB52983162908F00001308312AA
:10038000A80070080319C829A80D2810FF3FC2292A
:1003900083162A08F00001308312A900700803199F
:1003A000D529A90D2910FF3FCF2983162B08F0006E
:1003B00001308312AA0070080319E229AA0D2A103D
:1003C000FF3FDC2983162C08F00001308312AB00BC
:1003D00070080319EF29AB0D2B10FF3FE929831695
:1003E0002208F00001308312AE0070080319FC29C6
:1003F000AE0D2E10FF3FF62983162308F0000130C2
:100400008312B40070080319092AB40D3410FF3F99
:10041000032A83162408F00001308312AF0070080D
:100420000319162AAF0D2F10FF3F102A831621083B
:100430008312A200831621088312A30083162008CA
:100440008312AD00831621088400210884008001F6
:1004500080302104F00070088312A200700884002C
:10046000700884008001831621088312A2002D08E1
:1004700084000008F1002F082E04F0003408F00476
:10048000F0097108F0052D0884002D08840070081B
:10049000800080302D04F2007208AD0072088400E4
:1004A0000008F1002F082E04F0003408F004F009D1
:1004B0007108F005720884007208840070088000DA
:1004C0008030AD0630308316AE0085223030831682
:1004D000AE00852230308316AE0085223830831678
:1004E000AE00852208308316AE00852201308316C7
:1004F000AE00852206308316AE0085220C308316AE
:10050000AE0085220130AC000800031383122208DC
:10051000840022088400800100308316AE1B013065
:10052000F1007108003A0319A22A831223088400FB
:100530000008F0002408F004220884002208840047
:100540007008800003138312003083162E1B0130C5
:10055000F1007108003A0319BA2A831223088400B3
:100560000008F0002508F004220884002208840016
:10057000700880000313831200308316AE1A013016
:10058000F1007108003A0319D22A8312230884006B
:100590000008F0002608F0042208840022088400E5
:1005A0007008800003138312003083162E1A013066
:1005B000F1007108003A0319EA2A83122308840023
:1005C0000008F0002708F0042208840022088400B4
:1005D000700880000313831200308316AE190130B7
:1005E000F1007108003A0319022B831223088400DA
:1005F0000008F0002808F004220884002208840083
:100600007008800003138312003083162E19013006
:10061000F1007108003A03191A2B83122308840091
:100620000008F0002908F004220884002208840051
:10063000700880000313831200308316AE18013057
:10064000F1007108003A0319322B83122308840049
:100650000008F0002A08F004220884002208840020
:100660007008800003138312013083162E05F100F9
:100670007108003A0319492B8312230884000008EB
:10068000F0002B08F004220884002208840070087F
:100690008000031383122C08013A031D5E2B2D08E2
:1006A00084000008F1002E09F0007108F0052D0803
:1006B00084002D088400700880006A2B2D088400B7
:1006C0000008F0002E08F0042D0884002D08840096
:1006D000700880002D0884000008F0002F08F00446
:1006E0002D0884002D0884007008800088272D08BC
:1006F00084000008F1002F09F0007108F0052D08B2
:1007000084002D0884007008800088272C08013A96
:10071000031D8E2B8A15BD228A11912B8A151B234E
:100720008A1108008A1507238A110030F200F300AD
:10073000E830F4000330F500F601F7018A15DE21F8
:100740008A1170088316A6007108A7007208A80015
:100750007308A9002008F4002108F500F601F7014C
:10076000A52570088316A6007108A7007208A800C6
:100770007308A9000330F40074080319C62BF30CA6
:10078000F20CF10CF00CF313FF3FBD2B7008A4002A
:100790007108A5008A1507238A112208F40023088E
:1007A000F500F601F7010030F200F3008A15DE21B2
:1007B0008A1170088316AA007108AB007208AC0099
:1007C0007308AD002408F0002508F100F201F301E0
:1007D0000330F40074080319F42BF00DF10DF20D41
:1007E000F30D7010FF3FEB2B7008F4007108F5005B
:1007F0007208F6007308F7002A08F0002B08F100D1
:100800002C08F2002D08F300A52570088316A60019
:100810007108A7007208A8007308A9000A30F40044
:10082000F5012408F0002508F1008A1537228A1105
:1008300070088316A4007108A50000307102031D22
:10084000232C033070020318262C582C83123108F5
:10085000840083162908003C031D382C2808003C1E
:10086000031D382C2708003C031D382C2608003CAB
:100870000318552C83123208800483162408AE0016
:100880008A15AC228A118312330880058316240846
:10089000AE008A15AC228A110130A602031CA70201
:1008A000031CA802031CA902292C8312330880050B
:1008B000031383120800031383162308F00000308B
:1008C000F1007F307002F4000030031C013F710220
:1008D000F5007408A8007508A90080307506F000BE
:1008E00080307002031D762C0030740203189F2C98
:1008F000F401F501F601F7012008F0002108F100EC
:100900002208F2002308F3008A151C218A11FF3007
:1009100003180030F00070080319942C8316A4010A
:10092000A501A601A7019E2C031383160030A40085
:100930000030A5000030A6007F30A700F22C290867
:10094000003C031DA52C2808183C0318B02C2008D7
:10095000A4002108A5002208A6002308A700F22C65
:100960002008F0002108F1002208F2002308F3001B
:1009700041268A1515228A1170088316A400710871
:10098000A5007208A6007308A7002008F40021083B
:10099000F5002208F6002308F7008A151C218A11A9
:1009A000FF3003180030F00070080319F22C831692
:1009B0002408F0002508F1002608F2002708F300BB
:1009C0000030F4000030F5000030F6007F30F70012
:1009D000FD2470088316A4007108A5007208A60003
:1009E0007308A700031383162408F0002508F100FC
:1009F0002608F2002708F300080003138312720888
:100A00007606A100F801F90173087702031C202D76
:100A10007708FD007308F7007D08F3007608FD00F5
:100A20007208F6007D08F2007508FD007108F500F7
:100A30007D08F1007408FD007008F4007D08F000E6
:100A400077080319A12D7208FA00F217F617770834
:100A50007302F7000319532D08307702031C492D48
:100A6000F7007408F9007508F4007608F500F6013F
:100A700008307702031C492DF7007408F900750847
:100A8000F400F50108307702031C492D7A08F200C2
:100A9000A12D77080319532D0310F60CF50CF40C57
:100AA000F90CF70B4C2DA11F602DF909F409F5097C
:100AB000F609F90A0319F40A0319F50A0319F60AE3
:100AC0007908F80774080318740FF00775080318FD
:100AD000750FF10776080318760FF207A11B792D21
:100AE000031C892DF20CF10CF00CF80CF30F892D7E
:100AF0009B2D03188F2DF809F009F109F209F80A66
:100B00000319F00A0319F10A0319F20A8030FA06F0
:100B1000952D0130FC008A1561208A11A32D023029
:100B2000FC008A1561208A11A32D0430FC008A156F
:100B3000AD218A11A32D0830FC008A15F9228A11F3
:100B4000A32D0030FC000000080003138312FC01F9
:100B5000F71BFC0AFD01FB01FA01F901F80173081A
:100B60007204710470040319392E73087706B000FB
:100B7000B01BFD09F71FC72DF409F509F609F709A0
:100B8000F40A0319F50A0319F60A0319F70AF31F01
:100B9000D42DF009F109F209F309F00A0319F10A59
:100BA0000319F20A0319F30A73087704B000B01BA3
:100BB000F52D5020FC1B122EFD1F392EF009F109D6
:100BC000F209F309F00A0319F10A0319F20A0319E9
:100BD000F30AF809F909FA09FB09F80A0319F90AED
:100BE0000319FA0A0319FB0A392EF71F0C2EF31BFF
:100BF000062E7308FB007208FA007108F9007008ED
:100C0000F800F301F201F101F001DC2DF301F20132
:100C1000F101F001F00A0034F309F209F109F009D9
:100C2000FC17D92DF80A0319F90A0319FA0A03194E
:100C3000FB0A74087802031DDC2D75087902031D78
:100C4000DC2D76087A02031DDC2D77087B02031D5C
:100C5000DC2DFB01FA01F901F801F00A0319F10A90
:100C60000319F20A0319F30AF31FDC2DB001301641
:100C7000FF34B0017C1C3F2E8A15DD228A11003F13
:100C8000080003138312FB01FC01F8017308031928
:100C9000B92E7208FA00F2179E30F302F31FA92E44
:100CA000F309F30A08307302031C7E2EF300F80DDB
:100CB0007008F8007108F0007208F100F2010830C5
:100CC0007302031C7E2EF300F80D7008F800710803
:100CD000F000F10108307302031C7E2EF300F80DC2
:100CE0007008F800F00108307302031C7E2EF30038
:100CF000F80DF8017308031D0310882E73080319FB
:100D0000882E0310F20CF10CF00CF80CF30B812E72
:100D10007B1B781C962E031C962EF80A0319F00AEA
:100D20000319F10A0319F20AF21BB62EFA1FB92EA3
:100D3000F209F109F009F809F80A0319F00A031990
:100D4000F10A0319F20AB92EF201F101F001F801DA
:100D5000B92E7B14FB1FBC2EF201FA1FBC2EF20031
:100D6000F100F000F800FA0DF20CBC2E0130FC008E
:100D7000BE2E0030FC00BE2EFF30FC00FC08031924
:100D8000C42E8A15CE228A117208F3007108F2006F
:100D90007008F1007808F000080001300313831692
:100DA000A00083126E08003C031DD82E6D08093C7C
:100DB0000318DC2E8316A00A0313831683126E0811
:100DC000003C031DE52E6D08633C0318E92E8316D5
:100DD000A00A0313831683126E08033C031DF22E30
:100DE0006D08E73C0318F62E8316A00A031383163A
:100DF00083126E08273C031DFF2E6D080F3C03185D
:100E0000032F8316A00A0313831683126F0884002E
:100E100020308000840A8000840A8000840A8000D8
:100E2000840A8000840A8001840383162008003C21
:100E300003183E2F0A30F400F50183126D08F0000C
:100E40006E08F1008A1537228A117808F0007908B7
:100E5000F10030307007800084030A30F400F5019F
:100E60006D08F0006E08F1008A1537228A117008AB
:100E7000ED007108EE008316A003152F0800031380
:100E800083126D08013A031D482F8030ED005F2F5B
:100E90006D08023A031D4F2FC030ED005F2F6D0823
:100EA000033A031D562F9430ED005F2F6D08043A6E
:100EB000031D5D2FD430ED005F2F8030ED006E08F4
:100EC0006D07F000F0037008ED000130AC00700811
:100ED0008316AE008522AC018316A0012008831280
:100EE0006F0784000008F2007208003A0319842F8B
:100EF0008316200883126F07840000088316AE0053
:100F000085228316A00A6E2F01308312AC000800E0
:100F100000000800FF3FFF3FFF3FFF3FFF3FFF3F55
:100F2000FF3FFF3FFF3FFF3FFF3FFF3FFF3FFF3FD1
:100F3000FF3FFF3FFF3FFF3FFF3FFF3FFF3FFF3FC1
:100F4000FF3FFF3FFF3FFF3FFF3FFF3FFF3FFF3FB1
:100F5000FF3FFF3FFF3FFF3FFF3FFF3FFF3FFF3FA1
:100F6000FF3FFF3FFF3FFF3FFF3FFF3FFF3FFF3F91
:100F7000FF3FFF3FFF3FFF3FFF3FFF3FFF3FFF3F81
:100F8000FF3FFF3FFF3FFF3FFF3FFF3FFF3FFF3F71
:100F9000FF3FFF3FFF3FFF3FFF3FFF3FFF3FFF3F61
:100FA000FF3FFF3FFF3FFF3FFF3FFF3FFF3FFF3F51
:100FB000FF3FFF3FFF3FFF3FFF3FFF3FFF3FFF3F41
:100FC000FF3FFF3FFF3FFF3FFF3FFF3FFF3FFF3F31
:100FD000FF3FFF3FFF3FFF3FFF3FFF3FFF3FFF3F21
:100FE000FF3FFF3FFF3FFF3FFF3FFF3FFF3FFF3F11
:100FF000FF3FFF3FFF3FFF3FFF3FFF3FFF3FFF3F01
:1010000003138312FB017308031D77080319572884
:1010100072087606FA007708F3077E30031C14285E
:10102000F30203185A281728F302031C5D287208DC
:10103000F8007108FC007008FD00F817F61703109F
:10104000F201F101F0011830A1007D1C3128740873
:10105000F00775080318750FF10776080318760F67
:10106000F207F20CF10CF00CF80CFC0CFD0C031068
:10107000A10B2528F21B4128F80DF00DF10DF20D02
:10108000F3037B1B701C5328F81F5328F00A031925
:10109000F10A0319F20A031D5328F20CF10CF00CAB
:1010A000F30A03195A28FA1FF21300305F2801309F
:1010B00012235F280230F9225F280430EB2200005F
:1010C0000800031383127C189928FC186A287C19DD
:1010D000B8286328A1017208031D8A287108F2004C
:1010E0007008F1007808F000F801A1157208031DDE
:1010F0008A287108F2007008F100F001A111211690
:101100007208031D8A287108F200F101A115720806
:101110000319AC282108F302031D031CB028031097
:10112000F21B9928F80DF00DF10DF20DF30B90283C
:10113000B0287B1B701CB428F81FB428F00A0319D0
:10114000F10A0319F20A031DB428F20CF10CF00C99
:10115000F30A0319B828B4280130FC001223BB2875
:101160000230FC00EB22BB280430FC002A23BB2801
:101170000830FC00F9220000080003138312FB0171
:10118000FC01FA0173080319FC28F2178E30F302F0
:10119000F31BCD280319CD28FF28F309F30A0830E3
:1011A0007302031CE228F300F10D7208F100F20152
:1011B00008307302031CE228F10DF1017308031DCE
:1011C0000310EA2873080319EA280310F20CF10C43
:1011D000F30BE5287B1B711CF428031CF428F10A8F
:1011E0000319F20AF21B0B29FA1F0E29F209F10961
:1011F000F10A0319F20A0E29F201F1010E297B14FA
:10120000FB1F1129F201FA1F1129FF30F200F10032
:10121000FA0DF20C11290130FC0013290030FC00FA
:101220001329FF30FC00FC0803191729CE2271088E
:10123000F0007208F100080003138312FA0173082A
:10124000031D7A147708031DFA147A080319682914
:10125000033A031933297A183029F61F66296429BD
:10126000F21F6429662972088039FA00F2137608A1
:101270008039F6137A06031941297A08031964297B
:1012800066297708730203194829031C5C29602921
:101290007608720203194F29031C5C29602975081E
:1012A000710203195629031C5C2960297408700215
:1012B0000319682903186029FA08031966296429A3
:1012C000FA080319642966290314080003100800AA
:1012D0000314031508000800031383129F01C03094
:1012E0009F04403083161F04F00070089F00803078
:1012F00070049F0083126D08F000F00D7010F00D67
:101300007010F00D701070089F041F1423231F1518
:101310001F08F200003072190130F2007208013A21
:10132000031D9429000088291E08F200F3017208A9
:10133000F300F2017208EE007308EF0083161E0836
:1013400072048312EE007308EF000030EF041F10E8
:101350006E08F0006F08F100080003138312A1016A
:101360007208031DC4297108F2007008F100F00131
:10137000A1157208031DC4297108F200F101A11121
:10138000211672080319D2292108F302031D031C38
:10139000D6290310F21BDA29F00DF10DF20DF30B33
:1013A000CA29D6290130FC001223DD290230FC00B5
:1013B000EB22DD290430FC002A23080003138312EA
:1013C0002230FC00F801F901FA01FB01FC030319CA
:1013D000142A0310FB0CFA0CF90CF80CF30CF20CA9
:1013E000F10CF00C031CE629FC030319062A74080F
:1013F000F80775080318750FF90776080318760FB4
:10140000FA0777080318770FFB07EA297408F8072B
:1014100075080318750FF90776080318760FFA0791
:1014200077080318770FFB0708000313831270086F
:10143000F8007108F0007208F1007308F200F3017F
:10144000FB01FC019E30F300FA01F21F332AF80978
:10145000F009F109F209F80A0319F00A0319F10A6F
:101460000319F20AFA170230FC0061200800031386
:101470008312F801F9011030FC00710DF80DF90D1F
:101480007408F8027508031C750FF90203184F2A37
:101490007408F80775080318750FF9070310F00DA5
:1014A000F10DFC0B3D2A0800031383126D08B100F7
:1014B0006E08F1000130F00071080319632AF00D85
:1014C0007010FF3F5D2A7008B200F0097008B30089
:1014D0006D08840070088005841770088005080076
:1014E000031383127008F8007108F000F101F20193
:1014F000F301FB01FC019630F300FA017008F100E2
:101500007808F000F801F201AD21080003138312FE
:1015100073087706031D992A72087606031D992A17
:1015200071087506031D992A7008740603190315BE
:101530000800031108000800031383127008F80064
:10154000FB01FC019E30F300FA01F201F101F00110
:101550000230FC006120080003138316AE03AE03C3
:101560002E08003C0318B92AAE030000000000005A
:10157000B02A0000000000000800083003138312A6
:10158000FB00FF30FA00FB0BC62AC92AFA0BC62A59
:10159000C32A1E30FA00FA0BCB2A08000313831269
:1015A0007B14FB1FDB2AF201FA1FFF30F200F1006F
:1015B000F000FA0DF20CFF30080003138312FB0950
:1015C000FA09F909F809F80A0319F90A0319FA0AD4
:1015D0000319FB0A0800031383127B15FB1FF72A6C
:1015E0000130F300F201F101F001FA0DF20CFF30CD
:1015F000080003138312FB14FB1F052BFF30F300BD
:10160000F200F100F000FA0DF20CFF300800A030FB
:1016100003138316AE000F30AF002E08F0002F0822
:10162000F100080003138312F201F101F001F80147
:10163000F30100300800103003138312FA00FA0B94
:101640001F2B00000800073003138312FA00FA0B67
:10165000272B080003138312FA1FF213003008002F
:10166000FF3FFF3FFF3FFF3FFF3FFF3FFF3FFF3F8A
:10167000FF3FFF3FFF3FFF3FFF3FFF3FFF3FFF3F7A
:10168000FF3FFF3FFF3FFF3FFF3FFF3FFF3FFF3F6A
:10169000FF3FFF3FFF3FFF3FFF3FFF3FFF3FFF3F5A
:1030000003138316870188018601073089003F304A
:1030100085008312860183160614831287018316A6
:10302000810190308B0007308312ED000630EE00F6
:103030000A1254220A1607308316A0000830A10095
:103040000230A2000130A300A4010730A500063021
:10305000A6000530A7000430A8000330A900023004
:10306000AA000130AB00AC018A110A127E218A1538
:103070000A160130ED000130EE004130E0006B3007
:10308000E1006B30E2007530E300E4016030EF00F6
:103090008A110A123F278A150A160230ED00013004
:1030A000EE004230E0006130E1006C30E20061305F
:1030B000E3006E30E4006330E5006530E600723016
:1030C000E700E8016030EF008A110A123F278A15F5
:1030D0000A160B30FC00FF30FB00FF30FA00FC0B3F
:1030E00072287928FB0B75287828FA0B7528722826
:1030F0006F283330FB00FF30FA00FB0B8028832859
:10310000FA0B80287D288830FA00FA0B85280716EC
:10311000A0013F30B50041309F00813083169F00F1
:1031200001308312ED000130EE004630E0006530E2
:10313000E1007330E2007A30E3003A30E400E50168
:103140006030EF008A110A123F278A150A162008FC
:10315000013A031DAC287429ED010A126C210A16EC
:103160000A1270220A167008E9007108EA00720853
:10317000EB007308EC006908B6006A08B7006B083A
:10318000B8006C08B9004130FB00FF30FA00FB0BBF
:10319000CA28CD28FA0BCA28C728C330FA00FA0B70
:1031A000CF2800003E08F0003F08F1000A1270220C
:1031B0000A167008BA007108BB007208BC007308D8
:1031C000BD006908F0006A08F1006B08F2006C08A5
:1031D000F3001930F4000430F5001630F6007E30AC
:1031E000F7000A1200200A160A12BD200A165830EB
:1031F000F00702300318013FF1077008BE007108A4
:10320000BF000A1270220A1670088316A000710807
:10321000A1007208A2007308A3008A110A125B249D
:103220008A150A160A12BD200A167008BE00710817
:10323000BF007008ED007108EE004030EF008A1109
:103240000A12CD268A150A1683123E08F0003F089E
:10325000F1000A1270220A167008F4007108F500D5
:103260007208F6007308F7003A08F0003B08F10016
:103270003C08F2003D08F3000A1286220A16FF30CD
:10328000031D0030F000700803194729A7280230F9
:10329000ED000130EE004030EF008A110A123F27A6
:1032A0008A150A160230ED000630EE006D30E0009F
:1032B0005630E1002030E200E3016030EF008A1177
:1032C0000A123F278A150A168230FB00FF30FA00E7
:1032D000FB0B6B296E29FA0B6B2968298730FA00E2
:1032E000FA0B70290000A7283608F0003708F10013
:1032F0003808F2003908F300EC30F4005130F500E2
:103300003830F6007D30F7000A1200200A167008E7
:10331000E9007108EA007208EB007308EC007030F5
:10332000F0000130F1000A1270220A166908F40058
:103330006A08F5006B08F6006C08F7008A110A129B
:10334000FD248A150A167008C6007108C7007208A5
:10335000C8007308C90001308316AE008A110A1232
:1033600085228A150A160130ED000130EE00493041
:10337000E0006E30E1006430E2006930E300743058
:10338000E4006130E5007330E600E7016030EF00F3
:103390008A110A123F278A150A160D30FC00FF30E9
:1033A000FB00FF30FA00FC0BD629DD29FB0BD929E5
:1033B000DC29FA0BD929D629D329BF30FB00FF30ED
:1033C000FA00FB0BE429E729FA0BE429E1292C3068
:1033D000FA00FA0BE92901308316AE008A110A12AD
:1033E00085228A150A16CA01CA0A2008003A031D56
:1033F000152A861206128611061186108713871267
:10340000F0010A129C220A167008BA007108BB006B
:103410007208BC007308BD0001308316AE008A112B
:103420000A1285228A150A16882801303505F4000B
:103430007408013A031D432A0530ED000A126C217D
:103440000A167008CB007108CC000A1270220A1606
:103450007008F4007108F5007208F6007308F700B0
:103460004608F0004708F1004808F2004908F30058
:103470000A121C210A16FF30031C0030F0007008ED
:103480000319432A35100030B5180130F4007408D0
:10349000013A031D722A0430ED000A126C210A164B
:1034A0007008CD007108CE000A1270220A1670084A
:1034B000F4007108F5007208F6007308F70046087A
:1034C000F0004708F1004808F2004908F3000A122A
:1034D0001C210A16FF30031C0030F000700803198D
:1034E000722AB510003035190130F4007408013A21
:1034F000031DA12A0730ED000A126C210A1670087C
:10350000CF007108D0000A1270220A167008F40069
:103510007108F5007208F6007308F7004608F0001D
:103520004708F1004808F2004908F3000A121C217C
:103530000A16FF30031C0030F00070080319A12A9E
:1035400035110030B5190130F4007408013A031D3B
:10355000D02A0630ED000A126C210A167008D1003C
:103560007108D2000A1270220A167008F40071085D
:10357000F5007208F6007308F7004608F0004708E7
:10358000F1004808F2004908F3000A121C210A164B
:10359000FF30031C0030F00070080319D02AB51169
:1035A0000030351A0130F4007408013A031DFF2A77
:1035B0000230ED000A126C210A167008D30071085F
:1035C000D4000A1270220A167008F4007108F5007F
:1035D0007208F6007308F7004608F0004708F1008B
:1035E0004808F2004908F3000A121C210A16FF30AD
:1035F000031C0030F00070080319FF2A3512003058
:10360000B51A0130F4007408013A031D2E2B013065
:10361000ED000A126C210A167008D5007108D60058
:103620000A1270220A167008F4007108F500720878
:10363000F6007308F7004608F0004708F100480854
:10364000F2004908F3000A121C210A16FF30031C7D
:103650000030F000700803192E2BB51201308316CC
:10366000AE008A110A1285228A150A160130350524
:10367000F4007408013A031DA32B4B08F0004C081A
:10368000F1000A1270220A164E30F4006230F50082
:103690005030F6007F30F7000A1200200A1670083A
:1036A000BA007108BB007208BC007308BD00700846
:1036B0008316A0007108A1007208A2007308A3007D
:1036C0008A110A125B248A150A160A12BD200A16EC
:1036D0007008CB007108CC007008ED007108EE0096
:1036E0005730EF008A110A12CD268A150A160130CA
:1036F0008312ED000230EE005730EF008A110A12FB
:103700003F278A150A160130ED000130EE003130F6
:10371000E0003A30E100E2016030EF008A110A1265
:103720003F278A150A160130ED000730EE006D3094
:10373000E0005630E100E2016030EF008A110A1229
:103740003F278A150A1601303505F4007408003A3F
:10375000031DC42B0130ED000130EE003130E000DC
:103760003A30E1002030E2004B30E3006530E40005
:103770007330E5007A30E600E7016030EF008A112F
:103780000A123F278A150A160030B5180130F400D6
:103790007408013A031D322C4D08F0004E08F10068
:1037A0000A1270220A164E30F4006230F5005030D2
:1037B000F6007F30F7000A1200200A167008BA00DF
:1037C0007108BB007208BC007308BD007008831646
:1037D000A0007108A1007208A2007308A3008A115A
:1037E0000A125B248A150A160A12BD200A167008EE
:1037F000CD007108CE007008ED007108EE00403079
:10380000EF008A110A12CD268A150A160230831299
:10381000ED000230EE004030EF008A110A123F271F
:103820008A150A160230ED000130EE003230E00059
:103830003A30E100E2016030EF008A110A123F27BE
:103840008A150A160230ED000730EE006D30E000F8
:103850005630E100E2016030EF008A110A123F2782
:103860008A150A160030B5180130F4007408003AC1
:10387000031D542C0230ED000130EE003230E00028
:103880003A30E1002030E2004B30E3006530E400E4
:103890007330E5007A30E600E7016030EF008A110E
:1038A0000A123F278A150A160D30FC00FF30FB0074
:1038B000FF30FA00FC0B5D2C642CFB0B602C632C9E
:1038C000FA0B602C5D2C5A2CBF30FB00FF30FA0045
:1038D000FB0B6B2C6E2CFA0B6B2C682C2C30FA002B
:1038E000FA0B702C01308316AE008A110A12852261
:1038F0008A150A16003035190130F4007408013AAF
:10390000031DE82C4F08F0005008F1000A12702245
:103910000A164E30F4006230F5005030F6007F3069
:10392000F7000A1200200A167008BA007108BB00DE
:103930007208BC007308BD0070088316A0007108EF
:10394000A1007208A2007308A3008A110A125B2466
:103950008A150A160A12BD200A167008CF007108CF
:10396000D0007008ED007108EE005730EF008A11AA
:103970000A12CD268A150A1601308312ED00023094
:10398000EE005730EF008A110A123F278A150A16F7
:103990000130ED000130EE003330E0003A30E1005C
:1039A000E2016030EF008A110A123F278A150A16D9
:1039B0000130ED000730EE006D30E0005630E100E0
:1039C000E2016030EF008A110A123F278A150A16B9
:1039D000003035190130F4007408003A031D0A2D37
:1039E0000130ED000130EE003330E0003A30E1000C
:1039F0002030E2004B30E3006530E4007330E50036
:103A00007A30E600E7016030EF008A110A123F27A2
:103A10008A150A160030B5190130F4007408013A0D
:103A2000031D782D5108F0005208F1000A1270228F
:103A30000A164E30F4006230F5005030F6007F3048
:103A4000F7000A1200200A167008BA007108BB00BD
:103A50007208BC007308BD0070088316A0007108CE
:103A6000A1007208A2007308A3008A110A125B2445
:103A70008A150A160A12BD200A167008D1007108AC
:103A8000D2007008ED007108EE004030EF008A119E
:103A90000A12CD268A150A1602308312ED00023072
:103AA000EE004030EF008A110A123F278A150A16ED
:103AB0000230ED000130EE003430E0003A30E10039
:103AC000E2016030EF008A110A123F278A150A16B8
:103AD0000230ED000730EE006D30E0005630E100BE
:103AE000E2016030EF008A110A123F278A150A1698
:103AF0000030B5190130F4007408003A031D9A2D06
:103B00000230ED000130EE003430E0003A30E100E8
:103B10002030E2004B30E3006530E4007330E50014
:103B20007A30E600E7016030EF008A110A123F2781
:103B30008A150A160D30FC00FF30FB00FF30FA003A
:103B4000FC0BA32DAA2DFB0BA62DA92DFA0BA62D40
:103B5000A32DA02DBF30FB00FF30FA00FB0BB12DD1
:103B6000B42DFA0BB12DAE2D2C30FA00FA0BB62D78
:103B700001308316AE008A110A1285228A150A16B0
:103B80000030351A0130F4007408013A031D2E2E5E
:103B90005308F0005408F1000A1270220A164E3041
:103BA000F4006230F5005030F6007F30F7000A1262
:103BB00000200A167008BA007108BB007208BC0029
:103BC0007308BD0070088316A0007108A100720878
:103BD000A2007308A3008A110A125B248A150A1630
:103BE0000A12BD200A167008D3007108D4007008AC
:103BF000ED007108EE005730EF008A110A12CD2651
:103C00008A150A1601308312ED000230EE0057309B
:103C1000EF008A110A123F278A150A160130ED00BB
:103C20000130EE003530E0003A30E100E201603072
:103C3000EF008A110A123F278A150A160130ED009B
:103C40000730EE006D30E0005630E100E2016030F8
:103C5000EF008A110A123F278A150A160030351A1A
:103C60000130F4007408003A031D502E0130ED00BD
:103C70000130EE003530E0003A30E1002030E20063
:103C80004B30E3006530E4007330E5007A30E60045
:103C9000E7016030EF008A110A123F278A150A16E1
:103CA0000030B51A0130F4007408013A031DBE2E2D
:103CB0005508F0005608F1000A1270220A164E301C
:103CC000F4006230F5005030F6007F30F7000A1241
:103CD00000200A167008BA007108BB007208BC0008
:103CE0007308BD0070088316A0007108A100720857
:103CF000A2007308A3008A110A125B248A150A160F
:103D00000A12BD200A167008D5007108D600700886
:103D1000ED007108EE004030EF008A110A12CD2646
:103D20008A150A1602308312ED000230EE00403090
:103D3000EF008A110A123F278A150A160230ED0099
:103D40000130EE003630E0003A30E100E201603050
:103D5000EF008A110A123F278A150A160230ED0079
:103D60000730EE006D30E0005630E100E2016030D7
:103D7000EF008A110A123F278A150A160030B51A79
:103D80000130F4007408003A031DE02E0230ED000B
:103D90000130EE003630E0003A30E1002030E20041
:103DA0004B30E3006530E4007330E5007A30E60024
:103DB000E7016030EF008A110A123F278A150A16C0
:103DC0000D30FC00FF30FB00FF30FA00FC0BE92E49
:103DD000F02EFB0BEC2EEF2EFA0BEC2EE92EE62E3E
:103DE000BF30FB00FF30FA00FB0BF72EFA2EFA0B68
:103DF000F72EF42E2C30FA00FA0BFC2E4A08143A57
:103E0000031D482F8612061286110611861087138D
:103E100001308316AE008A110A1285228A150A160D
:103E20000130ED000130EE005330E0007A30E10067
:103E30007530E2006E30E3006530E4007430E50078
:103E4000E6016030EF008A110A123F278A150A1630
:103E50004D30FC00FF30FB00FF30FA00FC0B312F2F
:103E6000382FFB0B342F372FFA0B342F312F2E2FF7
:103E70007E30FB00FF30FA00FB0B3F2F422FFA0B86
:103E80003F2F3C2F0D30FA00FA0B442F0000CA01DF
:103E900001303505F4007408003A031D512F8612D5
:103EA000522F86160030B5180130F4007408003A1D
:103EB000031D5C2F06125D2F0616003035190130E8
:103EC000F4007408003A031D672F8611682F8615C9
:103ED0000030B5190130F4007408003A031D722F48
:103EE0000611732F06150030351A0130F4007408DE
:103EF000003A031D7D2F86107E2F86140030B51AE0
:103F00000130F4007408003A031D882F8713892FAD
:103F100087173508003A031D9C2FB8308316A00080
:103F20000130A100E830A2000330A3008A110A1278
:103F300092238A150A168716F4299D2FFF3FFF3F0B
:02400E003A3F37
:00000001FF
